:100000000629A0008417800484138E010C1C8E0026
:100010002320031901292320031901292320012961
:10002000A0008F200C080D0403190129FB20841364
:100030002008800664001C281D288C0A03198D0FD7
:100040001A288006012920088E0601308C008D01B7
:10005000000820050E06031D08008C0A03198D0FE9
:100060002828080064004220031832284D20083058
:100070008F004E2042208E0C3D288F0B39284E20B9
:100080000E080800220884002008841780048413C6
:1000900000051F192006FF3E08001F171F0D063917
:1000A0008C005C208D008C0A5C201F1FB0281F1361
:1000B0008C000230C720B02800308A000C0882076C
:1000C000013475340334153400343C340C34D934E1
:1000D0008F00220884002009902084138F080319C0
:1000E0000129F03091000E0880389000F030910323
:1000F0000319910003198F03031901297F28932005
:1001000003010C1820088E1F20088E080319030114
:10011000900F8C28800673288D2800007628FF3ADF
:100120008417800501290D080C0403198C0A8030FE
:100130000C1A8D060C198D068C188D060D0D8C0D64
:100140008D0D01298F018E00FF308E07031C8F0754
:10015000031C012903308D00DF30B020A4288D015D
:10016000E83E8C008D09FC30031CB9288C0703186D
:10017000B6288C0764008D0FB6280C18BF288C1C7D
:10018000C3280000C328080003108D0C8C0CFF3E10
:100190000318C4280C0801298E000430CF289400CD
:1001A0000F080D02031DD6280E080C020430031898
:1001B0000130031902301405031DFF30012991019C
:1001C0009001103092000D0D900D910D0E089002CF
:1001D0000F08031C0F0F91020318F5280E08900753
:1001E0000F0803180F0F910703108C0D8D0D920B44
:1001F000E3280C0801298C098D098C0A03198D0A42
:10020000080083130313831264000800831602306E
:1002100085000130860083120612831606128312AF
:100220000613831606138312861283168612831210
:100230008610831686108312061183160611831208
:1002400086118316861105308312A2000830A000A3
:1002500073308E000A30682032308E000A306820F9
:100260000630A2000130A00004309F0032205A3C2A
:10027000031D36293220A80064002808413C031DD4
:100280004C29E52124088C0025088D008F010830B9
:10029000CC20031D30298D2164002808423C031D19
:1002A0005229C32164002808433C031D5829B22168
:1002B00064002808443C031D5E29D42164002808FA
:1002C000453C031D6F290530A2000830A0007330A3
:1002D0008E000A30682032308E000A3068206400B8
:1002E0002808463C031D8C29061283160612831229
:1002F0000613831606138312861283168612831240
:100300008610831686108312061183160611831237
:10031000861183168611831230290616831606125B
:10032000831206178316061383128614831686100B
:100330008312061583160611831201308F00F430E4
:10034000A3200612831606128312061383160613C1
:1003500083128610831686108312061183160611E7
:1003600083120800061683160612831206178316D8
:10037000061383128614831686108312861583163D
:10038000861183120800061683160612831286163B
:10039000831686128312861483168610831286159E
:1003A000831686118312080006168316061283121E
:1003B000861683168612831286148316861083127D
:1003C0000615831606118312080001308C008D017A
:1003D000053084000130102001308C00053084008D
:1003E000023001200C08A6000D08A70026088C008A
:1003F00027088D000F308E008F01DF20A4000D082C
:0C040000A5000A30A22008006300042AB6
:02400E00F53F7C
:00000001FF
